:020000040800F2
:1000000048130020890100089B2A0008D92700080E
:10001000512A0008550500089D3200080000000024
:100020000000000000000000000000005D2C00083F
:1000300095050008000000009F2A00085F2C0008BA
:10004000A3010008A3010008A3010008A301000800
:10005000A3010008A3010008A3010008A3010008F0
:10006000A3010008A3010008A3010008A3010008E0
:10007000A3010008A301000859050008A301000816
:10008000A3010008A3010008A3010008A3010008C0
:10009000A3010008A3010008A3010008A3010008B0
:1000A000A3010008D12C0008A3010008A301000847
:1000B000A3010008E12C0008A3010008A301000827
:1000C000A3010008A3010008A3010008A301000880
:1000D000A30100088D320008A3010008A301000855
:1000E000A3010008A3010008A301000800F002F822
:1000F00000F03AF80AA090E8000C82448344AAF188
:100100000107DA4501D100F02FF8AFF2090EBAE885
:100110000F0013F0010F18BFFB1A43F0010318473B
:100120007C4500009C450000103A24BF78C878C187
:10013000FAD8520724BF30C830C144BF04680C60ED
:10014000704700000023002400250026103A28BF35
:1001500078C1FBD8520728BF30C148BF0B60704739
:100160001FB51FBD10B510BD00F0D1F81146FFF747
:10017000F7FF03F011FB00F0EFF803B4FFF7F2FF15
:1001800003BC03F0EDF80000094880470948004728
:10019000FEE7FEE7FEE7FEE7FEE7FEE7FEE7FEE737
:1001A000FEE7FEE704480549054A064B7047000094
:1001B000CD2C0008ED000008480D00204813002059
:1001C000480F0020480F002070477047032A40F274
:1001D000308010F0030C00F0158011F8013BBCF1E9
:1001E000020F624498BF11F801CB00F8013B38BF01
:1001F00011F8013BA2F1040298BF00F801CB38BF0F
:1002000000F8013B11F0030300F04F80083AC0F002
:10021000088051F8043B083A51F804CBA0E80810D4
:10022000F5E7121D5CBF51F8043B40F8043BAFF307
:100230000080D20724BF11F8013B11F801CB48BF61
:1002400011F8012B24BF00F8013B00F801CB48BF97
:1002500000F8012B70474FF0000200B5134694469A
:100260009646203922BFA0E80C50A0E80C50B1F10E
:100270002001BFF4F7AF090728BFA0E80C5048BF22
:100280000CC05DF804EB890028BF40F8042B08BFC0
:10029000704748BF20F8022B11F0804F18BF00F8BC
:1002A000012B704770477047704710B5203AC0F077
:1002B0000B80B1E81850203AA0E81850B1E8185067
:1002C000A0E81850BFF4F5AF5FEA027C24BFB1E8A4
:1002D0001850A0E8185044BF18C918C0BDE8104015
:1002E0005FEA827C24BF51F8043B40F8043B08BF1E
:1002F0007047D20728BF31F8023B48BF11F8012BE5
:1003000028BF20F8023B48BF00F8012B7047754614
:1003100000F028F8AE4605006946534620F0070075
:10032000854618B020B5FFF73DFFBDE820404FF0EF
:1003300000064FF000074FF000084FF0000B21F0CF
:100340000701AC46ACE8C009ACE8C009ACE8C0099C
:10035000ACE8C0098D4670470446AFF300802046E4
:10036000FFF70BFF00487047E80C00207CB50446FF
:1003700010E053480068401C514908600846006876
:100380004FF6FF71884205DB00204D4908604D495A
:1003900003C97CBD01214C4800F0B0FC0028E8D125
:1003A000082C2DD2DFE804F004090E13181D2227B3
:1003B0000821012000F094F822E01821012000F02B
:1003C0008FF81DE02821012000F08AF818E038217C
:1003D000012000F085F813E04821012000F080F8AA
:1003E0000EE05821012000F07BF809E0682101208F
:1003F00000F076F804E07821012000F071F800BFE9
:1004000000BFFC2001900A23012201A92F4801F01E
:100410001EFA002001900A23012201A92B4801F0B5
:1004200016FA012001900A23012201A9274801F0B0
:100430000EFA0A2303226946244801F047F99DF881
:10044000000000049DF8011040EA01209DF8021010
:1004500008431F490860084600681E4908600846AE
:10046000006800F40000E0B108460068C04308607E
:1004700008460068C0F31600086008460068401C83
:10048000086008460068404208600846006803F0BB
:10049000DAFF0546104A114B03F0ECFF094A03C28C
:1004A0000AE00C48006803F0CEFF05460A4A0B4BF1
:1004B00003F0E0FF034A03C2024903C969E70000F1
:1004C0006400002050000020000C01406800002063
:1004D000480000204C00002085F90F270088433F8A
:1004E00013B582B004460EE017480068401C164958
:1004F0000860084600684FF6FF71884203DB002061
:10050000114908601FBD0121104800F0F7FB0028C9
:10051000EAD104F00F0040F0500001900A230122BC
:1005200001A90B4801F093F9002001900A23012250
:1005300001A9074801F08BF90A23012203A9044805
:1005400001F085F900BFDDE764000020000C0140E8
:100550006800002000BFFEE710B5024800F0EEF88A
:1005600010BD00009801002030B590F840500124E3
:10057000AC40C56B6C60046863604468102C04D1A7
:100580000468A2600468E16003E00468A160046894
:10059000E26030BD704772B600BFFEE70146084614
:1005A000024B33F8100002B290B27047C60200202E
:1005B00001460846024B33F8100002B290B2704771
:1005C0000602002030B5A0F11002D41702EB5474DB
:1005D000E410094D2B5DD41702EB5474E410A2EB28
:1005E000C4050124AC401C4014B101220A7001E092
:1005F00000220A7030BD0000F001002030B5024634
:10060000D41702EB5474E410094D2B5D0246D41745
:1006100002EB5474E410A2EBC4050124AC401C406E
:1006200014B101220A7001E000220A7030BD0000FE
:10063000FA0100200146002291F82100022808D08A
:100640000420886300BF002081F8200000BF012043
:1006500070470868006820F00E000B681860086892
:10066000006820F001000B68186091F8403001200C
:100670009840CB6B5860012081F8210000BF00201A
:1006800081F8200000BF1046E2E7000070B5044684
:10069000002594F82100022803D00420A06301253E
:1006A00048E02068006820F00E002168086020689B
:1006B000006820F00100216808601F492068884216
:1006C00001D1012026E01C4914312068884201D163
:1006D00010201FE0184928312068884201D1801578
:1006E00018E015493C312068884201D1801411E09E
:1006F000114950312068884202D14FF4803009E01E
:100700000D4964312068884202D14FF4801001E025
:100710004FF08070084908394860012084F82100B2
:1007200000BF002084F8200000BF606B10B120469D
:10073000616B8847284670BD0800024070B50446CA
:10074000E06B05682068066894F840100420884033
:100750002840002846D006F00400002842D0206837
:10076000006800F0200028B92068006820F004002C
:100770002168086057492068884201D1042027E099
:10078000544914312068884201D1402020E0514969
:1007900028312068884201D1001519E04D493C31CB
:1007A0002068884202D14FF4804011E0494950311D
:1007B0002068884202D14FF4802009E04549643125
:1007C0002068884202D14FF4800001E04FF0806041
:1007D000404908394860E06A00287AD02046E16A3A
:1007E000884776E094F84010022088402840A0B363
:1007F00006F0020088B32068006800F0200040B9CD
:100800002068006820F00A0021680860012084F850
:10081000210030492068884201D1022028E02D497A
:1008200014312068884201D1202021E02949283153
:100830002068884201D140151AE026493C312068E1
:10084000884202D14FF4005012E022495031206812
:10085000884203D14FF400300AE017E01D496431AB
:100860002068884202D14FF4001001E04FF0007080
:1008700018490839486000BF002084F8200000BFF4
:10088000A06A30B32046A16A884722E094F840105D
:10089000082088402840E0B106F00800C8B1206870
:1008A000006820F00E002168086094F840100120D4
:1008B0008840E16B48600120A06384F8210000BFFC
:1008C000002084F8200000BF206B10B12046216B6F
:1008D000884770BD080002400146002209B9012086
:1008E0007047164B0868C01A1423B0FBF3F0800061
:1008F000086412480838C863022081F8210008689B
:10090000026843F6F0708243D1E901031843CB68D3
:1009100018430B6918434B6918438B691843CB691B
:10092000184302430868026000208863012081F8B0
:100930002100002081F8200000BFD1E7080002401C
:100940002DE9F04104460D4616461F464FF00008BB
:1009500000BF94F82000012802D10220BDE8F081F8
:10096000012084F8200000BF94F8210001282CD138
:10097000022084F821000020A0632068006820F095
:100980000100216808603B46324629462046FFF7B1
:10099000EBFDE06A30B12068006840F00E0021688D
:1009A00008600BE02068006820F0040021680860FF
:1009B0002068006840F00A0021680860206800682C
:1009C00040F001002168086006E000BF002084F8C4
:1009D000200000BF4FF002084046BFE72DE9F8476E
:1009E0000346002294466EE14FF0010808FA02F433
:1009F000D1F8008008EA0400A0427DD1DFF8DCA233
:100A0000D1F80480A8EB0A09D0453AD014DCB8F13B
:100A1000030F50D009DCB8F1000F31D0B8F1010F4D
:100A20001CD0B8F1020F49D120E0B8F1110F18D055
:100A3000B8F1120F42D11EE0B9F5881F25D006DCAF
:100A4000B9F5803F20D0B9F5801F37D11AE0B9F54C
:100A5000001F18D0B9F5041F30D117E0D1F80CC031
:100A60002DE0D1F80C8008F1040C28E0D1F80C80BE
:100A700008F1080C23E0D1F80C8008F10C0C1EE002
:100A800000BF00BF00BF00BF00BF00BFD1F808809B
:100A9000B8F1000F02D14FF0040C0BE0D1F8088040
:100AA000B8F1010F03D14FF0080C1C6102E04FF0C8
:100AB000080C5C6103E04FF0000C00E000BF00BFD9
:100AC000FF2801D8984601E003F104084646FF28B4
:100AD00002D84FEA820803E0A2F108084FEA88082A
:100AE0004746D6F800804FF00F0909FA07F928EABF
:100AF00009080CFA07F900E088E048EA0908C6F896
:100B00000080D1F8048008F08058B8F1805F7DD172
:100B100000BFDFF8CC81D8F8188048F00108DFF872
:100B2000C091C9F81880C846D8F8188008F00108A4
:100B3000CDF8008000BF00BF4FEAB9384FEA9209F4
:100B400058F829504FEA82784FEA18794FF00F0889
:100B500008FA09F825EA0805DFF88881434502D13B
:100B60004FF0000816E0DFF88081434502D14FF0D6
:100B700001080FE0DFF87481434502D14FF002080D
:100B800008E0DFF86C81434502D14FF0030801E033
:100B90004FF004084FEA82794FEA197908FA09F808
:100BA00048EA0505DFF84C814FEA920948F82950D8
:100BB000D1F8048008F48018B8F5801F0AD1DFF856
:100BC0003881D8F8008048EA0008DFF82C91C9F88D
:100BD000008009E0DFF82081D8F8008028EA0008CA
:100BE000DFF81491C9F80080D1F8048008F40018E7
:100BF000B8F5001F10D1DFF8008108F10408D8F81B
:100C0000008048EA0008DFF8F09000E05AE009F1BF
:100C10000409C9F800800DE0DFF8DC8008F1040861
:100C2000D8F8008028EA0008DFF8CC9009F1040920
:100C3000C9F80080D1F8048008F40038B8F5003F06
:100C40000ED1DFF8B480A8F10408D8F8008048EA93
:100C50000008DFF8A490A9F10409C9F800800DE0AC
:100C6000DFF89480A8F10408D8F8008028EA00088A
:100C7000DFF88490A9F10409C9F80080D1F8048054
:100C800008F48038B8F5803F0ED1DFF86C80A8F109
:100C90000808D8F8008048EA0008DFF85C90A9F15D
:100CA0000809C9F800800DE0DFF84C80A8F10808B9
:100CB000D8F8008028EA0008DFF83C90A9F108097C
:100CC000C9F80080521CD1F8008028FA02F8B8F167
:100CD000000F7FF489AEBDE8F88700000000111016
:100CE0000010024000080140000C014000100140CB
:100CF00000140140080001400804014002469368C6
:100D00000B400BB1012000E00020704710B5C26815
:100D100021EA020302EA010443EA0443036110BD2D
:100D20000AB1016101E00B040361704701480068EA
:100D3000704700003000002003480068034909782C
:100D40000844014908607047300000203800002046
:100D500010B50848006840F01000064908600320FC
:100D600000F0A8F80F2000F007F800F02BF80020A2
:100D700010BD00000020024070B504460E48007807
:100D80004FF47A71B1FBF0F00C490968B1FBF0F552
:100D9000284600F05FFF08B1012070BD102C07D27B
:100DA00000222146501E00F047F80548046001E08B
:100DB0000120F2E70020F0E7380000203C0000208E
:100DC0003400002008B500BF1148806940F00100E0
:100DD0000F4988610846806900F00100009000BF5B
:100DE00000BF00BF0846C06940F08050C861084697
:100DF000C06900F08050009000BF00BF00BF0549EF
:100E0000486820F0E06040F00070486000BF08BD16
:100E1000001002400000014001460846002809DB9E
:100E200000F01F0301229A4043099B0003F1E023D5
:100E3000C3F8002100BF70472DE9F05F80460D46E2
:100E40001646002702F070FA074639462A4633460E
:100E500001F00700C0F1070ABAF1040F02D94FF000
:100E6000040A01E0C0F1070AD14600F1040ABAF110
:100E7000070F02D24FF0000A01E0A0F1030AD446A6
:100E80004FF0010A0AFA09FAAAF1010A0AEA020A6B
:100E90000AFA0CFA4FF0010B0BFA0CFBABF1010B49
:100EA0000BEA030B4AEA0B042146404602F044FADF
:100EB000BDE8F09F00BF00F00702064B19684FF62F
:100EC000FF031940044B0B4343EA0221014B196015
:100ED00000BF70470CED00E00000FA0570B5044655
:100EE0000D460CB9012070BD5A48006800F007009B
:100EF000A8420ED25748006820F007002843554901
:100F000008600846006800F00700A84201D00120F0
:100F1000E9E7207800F0020002281DD1207800F0D7
:100F20000400042805D14C48406840F4E0604A4978
:100F30004860207800F00800082805D1464840683D
:100F400040F46050444948604348406820F0F00055
:100F5000A168084340494860207800F0010078B358
:100F60006068012806D13C48006800F4003090B960
:100F70000120B8E76068022806D13748006800F011
:100F8000007040B90120AEE73348006800F002006D
:100F900008B90120A7E73048406820F003006168E5
:100FA00008432D494860FFF7C1FE064609E0FFF7F8
:100FB000BDFE801B41F28831884202D9032092E7AE
:100FC00007E02548406800F00C006168B0EB810F35
:100FD000EDD12048006800F00700A8420ED91D4856
:100FE000006820F0070028431A4908600846006896
:100FF00000F00700A84201D0012074E7207800F03B
:101000000400042807D11448406820F4E060E16837
:10101000084311494860207800F00800082808D1EA
:101020000D48406820F46050216940EAC1000A4937
:10103000486000F03FF808494968C1F30311074AC6
:10104000515CC8400649086006480068FFF794FEF6
:10105000002048E7002002400010024082460008BD
:101060003C00002034000020014800687047000068
:101070003C00002000B5FFF7F7FF04494968C1F3C1
:101080000221034A515CC84000BD0000001002402C
:101090009246000800B5FFF7E7FF04494968C1F32D
:1010A000C221034A515CC84000BD0000001002404C
:1010B0009246000870B50021002200240023002081
:1010C000134D696801F00C05F5B1042D02D0082D0F
:1010D00019D101E00F4819E00F4DC1F38346AB5D14
:1010E00001F4803555B10A4D6D68C5F340450B4E8E
:1010F000725D084D5D43B5FBF2F402E0084D03FB61
:1011000005F4204602E000BF024800BF00BF70BDEA
:101110000010024000127A00704600088046000865
:1011200000093D00F8B504460CB90120F8BD20784F
:1011300000F00100002878D0F848406800F00C006A
:1011400004280CD0F548406800F00C00082811D1A4
:10115000F248406800F48030B0F5803F0AD1EF4893
:10116000006800F4003000285FD0606800285CD17F
:101170000120DBE700BF6068B0F5803F06D1E7489B
:10118000006840F48030E549086028E0606858B99C
:10119000E248006820F48030E049086008460068B2
:1011A00020F4802008601AE06068B0F5A02F0BD111
:1011B000DA48006840F48020D84908600846006892
:1011C00040F4803008600AE0D448006820F48030A1
:1011D000D24908600846006820F48020086000BFFB
:1011E000606888B1FFF7A2FD054606E0FFF79EFDA7
:1011F000401B642801D9032098E7C848006800F420
:1012000000300028F2D010E0FFF790FD054606E020
:10121000FFF78CFD401B642801D9032086E7BF48F7
:10122000006800F400300028F2D1207800F00200BD
:10123000022857D1B948406800F00C0050B1B748B7
:10124000406800F00C00082818D1B448406800F449
:10125000803098B9B148006800F0020020B12069E0
:10126000012801D0012061E7AC48006820F0F800B7
:10127000616940EAC100A949086033E02069E8B12A
:101280000120A7490860FFF751FD054606E0FFF77A
:101290004DFD401B022801D9032047E79F48006805
:1012A00000F002000028F2D09C48006820F0F8000E
:1012B000616940EAC1009949086013E0002098493B
:1012C0000860FFF733FD054606E0FFF72FFD401BE2
:1012D000022801D9032029E79048006800F00200A5
:1012E0000028F2D1207800F0080008282DD1A0694C
:1012F000B8B101208B490860FFF718FD054606E0EC
:10130000FFF714FD401B022801D903200EE7834894
:10131000406A00F002000028F2D0012001F0C0FB7A
:1013200013E000207F490860FFF700FD054606E056
:10133000FFF7FCFC401B022801D90320F6E67748A2
:10134000406A00F002000028F2D1207800F004008A
:10135000042873D100277148C06900F0805070B92B
:1013600000BF6E48C06940F080506C49C8610846B3
:10137000C06900F08050009000BF00BF01276A489C
:10138000006800F48070B0B96748006840F480706D
:1013900065490860FFF7CAFC054606E0FFF7C6FC92
:1013A000401B642801D90320C0E65F48006800F4B0
:1013B00080700028F2D000BFE068012806D15748AD
:1013C000006A40F001005549086227E0E06858B91A
:1013D0005248006A20F00100504908620846006A3D
:1013E00020F00400086219E0E06805280BD14B48A2
:1013F000006A40F00400494908620846006A40F06B
:10140000010008620AE04548006A20F001004349F3
:1014100008620846006A20F00400086200BFE06825
:10142000A0B1FFF783FC054609E0FFF77FFC401BF6
:1014300041F28831884202D9032077E622E037481A
:10144000006A00F002000028EFD012E0FFF76EFC07
:10145000054608E0FFF76AFC401B41F288318842EC
:1014600001D9032062E62D48006A00F0020000283E
:10147000F0D1012F05D12948C06920F080502749BB
:10148000C86100BFE069C8B32448406800F00C00A0
:10149000082860D0E069022848D100202049086669
:1014A000FFF744FC054606E0FFF740FC401B02281E
:1014B00001D903203AE61948006800F000700028BE
:1014C000F2D1206AB0F5803F07D11448406820F47B
:1014D0000030A168084311494860D4E90801084375
:1014E0000E49496821F4741108430C4948600120F1
:1014F0000B490866FFF71AFC054607E03DE0FFF7D9
:1015000015FC401B022801D903200FE603480068A0
:1015100000F000700028F2D02FE000000010024020
:101520000000424280044242007000400020144902
:101530000866FFF7FBFB054606E0FFF7F7FB401BDD
:10154000022801D90320F1E50E48006800F0007080
:101550000028F2D111E0E069012800D1E6E5094850
:10156000466806F48031206A814204D106F4701185
:10157000606A814201D00120D8E50020D6E5000054
:10158000000042420010024010B504460CB9012090
:1015900010BD606A38B96068B0F5827F00D105E09F
:1015A0000021E16102E00021216161610021A1626D
:1015B00094F8510028B9002084F85000204600F02B
:1015C00043F8022084F851002068006820F04000B1
:1015D00021680860A08800F48270218901F4044128
:1015E0000843A18901F400610843217C01F0020154
:1015F0000843217D01F001010843218B01F40071B2
:101600000843217F01F0380108432021095D01F0E2
:1016100080010843218D01F40051084321680860CE
:101620000421A06901EA1040216848602068C0696F
:1016300020F400602168C86100206065012084F802
:1016400051000020A4E7000010B586B00446002039
:1016500002900390049005901949206888422DD18A
:1016600000BF1848806940F48050164988610846D8
:10167000806900F48050019000BF00BF00BF0846A1
:10168000806940F0040088610846806900F0040029
:10169000019000BF00BFB020029002200390032001
:1016A000059002A90848FFF799F940200290002010
:1016B0000390049002A90448FFF790F906B010BD0A
:1016C0000030014000100240000801402DE9F843BD
:1016D0000446884616461D4694F85100012802D05B
:1016E0000220BDE8F8836068B0F5827F0CD1A06865
:1016F00050B9042084F85100334642464146204602
:10170000009500F083F9ECE7FFF710FB0746B8F10E
:10171000000F00D00EB90120E3E700BF94F850009D
:10172000012801D10220DCE7012084F8500000BF2D
:10173000042084F8510000206065C4F83880A68732
:10174000E6872063A086E08620646064A068B0F528
:10175000004F0BD12068006820F04000216808602D
:101760002068006820F480402168086020680068D4
:1017700000F04000402805D02068006840F040009C
:1017800021680860E06830BB21E02068806800F0D4
:10179000010050B12068007BA16B0870A06B401C59
:1017A000A063E08F401EE08711E0FFF7BFFAC01B87
:1017B000A84201D3681C00B94DB9012084F851003A
:1017C00000BF002084F8500000BF032089E7E08FAD
:1017D0000028DAD125E021E02068806800F00100CF
:1017E00050B12068C068A16B0880A06B801CA0630A
:1017F000E08F401EE08711E0FFF798FAC01BA84277
:1018000001D3681C00B94DB9012084F8510000BF14
:10181000002084F8500000BF032062E7E08F00281A
:10182000DAD13A462946204601F04EF908B1202087
:101830006065012084F8510000BF002084F850004A
:1018400000BF606D08B101204BE7002049E72DE99A
:10185000F84304460F4616461D46FFF767FA8046D2
:10186000B14694F85100012802D00220BDE8F88367
:1018700007B10EB90120F9E700BF94F85000012824
:1018800001D10220F2E7012084F8500000BF0320BC
:1018900084F85100002060652763A686E686A06371
:1018A000A087E08760642064A068B0F5004F0BD18A
:1018B0002068006820F04000216808602068006807
:1018C00040F48040216808602068006800F0400013
:1018D000402805D02068006840F04000216808607A
:1018E000E068B0F5006F37D1606810B1B9F1010F51
:1018F00009D1206B00882168C860206B801C2063A0
:10190000E08E401EE08623E02068806800F0020040
:1019100002280AD1206B00882168C860206B801CD7
:101920002063E08E401EE08612E0FFF7FFF9A0EB97
:101930000800A84201D3681C00B94DB9012084F801
:10194000510000BF002084F8500000BF03208DE745
:10195000E08E0028D8D136E0606810B1B9F1010FEF
:1019600009D1206B007821680873206B401C20632C
:10197000E08E401EE08623E02068806800F00200D0
:1019800002280AD1206B007821680873206B401C64
:101990002063E08E401EE08612E0FFF7C7F9A0EB5F
:1019A0000800A84201D3681C00B94DB9012084F891
:1019B000510000BF002084F8500000BF032055E70D
:1019C000E08E0028D8D142462946204601F0B8F8DA
:1019D00008B120206065A06850B900BF00200090C9
:1019E0002068C068009020688068009000BF00BF39
:1019F000012084F8510000BF002084F8500000BF8F
:101A0000606D08B1012031E700202FE72DE9FE4F7E
:101A100004460F4690461D460C9E01200190FFF79C
:101A200085F9814694F851B060680290AA46BBF1EE
:101A3000010F0BD00298B0F5827F04D1A06810B9D5
:101A4000BBF1040F02D00220BDE8FE8F1FB1B8F138
:101A5000000F00D00DB90120F6E700BF94F8500048
:101A6000012801D10220EFE7012084F8500000BFD7
:101A700094F85100042802D0052084F85100002079
:101A80006065C4F83880E587A5872763E586A58665
:101A9000206460642068006800F04000402805D0A1
:101AA0002068006840F0400021680860E068B0F5F8
:101AB000006F52D1606810B1BAF1010F09D1206BEB
:101AC00000882168C860206B801C2063E08E401E67
:101AD000E0863BE02068806800F00200022810D118
:101AE000E08E70B1019801280BD1206B008821682D
:101AF000C860206B801C2063E08E401EE0860020C2
:101B000001902068806800F0010068B1E08F58B152
:101B10002068C068A16B0880A06B801CA063E08F68
:101B2000401EE08701200190FFF700F9A0EB0900BB
:101B3000B0420BD3701C48B1012084F8510000BFA3
:101B4000002084F8500000BF03207DE7E08E0028CD
:101B5000C0D1E08F0028BDD152E0606810B1BAF169
:101B6000010F09D1206B007821680873206B401C9D
:101B70002063E08E401EE0863CE02068806800F034
:101B80000200022810D1E08E70B1019801280BD11B
:101B9000206B007821680873206B401C2063E08E66
:101BA000401EE086002001902068806800F001005F
:101BB00068B1E08F58B12068C068A16B0870A06B55
:101BC000401CA063E08F401EE08701200190FFF7DA
:101BD000ADF8A0EB0900B04201D3701C00B94EB9BA
:101BE000012084F8510000BF002084F8500000BF9D
:101BF000032029E7E08E0028BFD1E08F0028BCD168
:101C00004A463146204600F09BFF40B120206065E7
:101C100000BF002084F8500000BF012014E7A06836
:101C200050B900BF002000902068C0680090206874
:101C30008068009000BF00BF012084F8510000BF01
:101C4000002084F8500000BF606D08B10120FBE661
:101C50000020F9E670B504462546681EB0F1807F85
:101C600001D301200FE0681E4FF0E02148610F21F1
:101C70004FF0FF3001F060FB00204FF0E021886161
:101C800007200861002070BD7047704730B50246DC
:101C90000B4600BF92F83C00012801D1022030BD64
:101CA000012082F83C0000BF022082F83D0010684D
:101CB00044681068816824F0700418680443106850
:101CC0004460104D1068A8420BD01068B0F1804FEE
:101CD00007D00D4D1068A84203D00C4D1068A842E3
:101CE00005D121F08001586801431068816001200E
:101CF00082F83D0000BF002082F83C0000BF00BF1A
:101D0000CDE70000002C0140000400400008004026
:101D100010B504460CB9012010BD94F83D0028B957
:101D2000002084F83C00204600F026F8022084F8C9
:101D30003D00211D206800F0DBFF012084F84600F3
:101D400000BF84F83E0001213F200155402001558D
:101D50004120015500BF00BF012084F8420043200C
:101D60000155442001554520015500BF012084F84C
:101D70003D000020D0E7000038B504461A4920682D
:101D8000884216D100BF1948806940F400601749A5
:101D900088610846806900F40060009000BF00BFC1
:101DA000002211461920FFF747F81920FFF734F8F1
:101DB00019E00F492068884215D100BF0B48C0695F
:101DC00040F002000949C8610846C06900F00200FD
:101DD000009000BF00BF002211461D20FFF72CF825
:101DE0001D20FFF719F838BD002C014000100240FB
:101DF00000040040014691F83D00012801D0012077
:101E00007047022081F83D000868C06840F001007A
:101E10000B68D860124B086898420BD00868B0F184
:101E2000804F07D00F4B0868984203D00E4B0868CC
:101E300098420CD10868806800F00702062A0CD08E
:101E40000868006840F001000B68186005E0086849
:101E5000006840F001000B6818600020D0E7000027
:101E6000002C0140000400400008004001460868C2
:101E7000C06820F001000A68D06000BF0868006AEE
:101E800041F21112104050B90868006A92101040D7
:101E900028B90868006820F001000A68106000BFD7
:101EA000012081F83D00002070472DE9F0410446F3
:101EB0000D46002700BF94F83C00012802D1022003
:101EC000BDE8F081012084F83C0000BF022084F8C6
:101ED0003D002068866826F0770626F47F46206855
:101EE00086602868502833D00CDC202850D004DCD1
:101EF00000284BD0102851D149E0302849D0402843
:101F00004CD139E060282DD0702807D0B0F5805F23
:101F100003D0B0F5005F41D10DE041E0D5E90213F7
:101F20006A68206800F026FF2068866846F0770619
:101F30002068866034E0D5E902136A68206800F002
:101F400019FF2068806840F480402168886027E09D
:101F5000EA686968206800F021FF5021206800F0DD
:101F600014FF1DE0EA686968206800F02AFF60211C
:101F7000206800F00AFF13E0EA686968206800F052
:101F80000DFF4021206800F000FF09E000BF00BF06
:101F900000BF2968206800F0F8FE01E0012700BFBB
:101FA00000BF012084F83D0000BF002084F83C0001
:101FB00000BF384684E7704770B504462068C5689E
:101FC0002068066906F00200022819D105F0020017
:101FD000022815D1401F2168086101202077206860
:101FE000806900F0030018B12046FFF7E4FF05E028
:101FF000204600F097F8204600F095F80020207762
:1020000006F00400042819D105F00400042815D1B5
:10201000C04321680861022020772068806900F4AD
:10202000407018B12046FFF7C6FF05E0204600F0DB
:1020300079F8204600F077F80020207706F00800B5
:10204000082819D105F00800082815D1C0432168D7
:102050000861042020772068C06900F0030018B1EF
:102060002046FFF7A8FF05E0204600F05BF8204679
:1020700000F059F80020207706F01000102819D140
:1020800005F01000102815D1C04321680861082010
:1020900020772068C06900F4407018B12046FFF72F
:1020A0008AFF05E0204600F03DF8204600F03BF8AE
:1020B0000020207706F0010048B105F0010030B1A2
:1020C0006FF0010021680861204600F02DF806F04D
:1020D0008000802809D105F08000802805D1C04308
:1020E000216808612046FFF7CFFD06F04000402838
:1020F00009D105F04000402805D1C043216808619E
:10210000204600F085F806F02000202809D105F0CF
:102110002000202805D1C043216808612046FFF730
:10212000B4FD70BD7047704710B504462C4884421A
:102130003AD101202B4908602B480068401C2A49ED
:10214000086008460068012805DD0120274908606D
:1021500000202549086026480068401C2449086082
:1021600008460068042805DD012022490860002097
:102170001F49086020480068401C1F490860084645
:102180000068B0F57A7F0FDB4FF400511B48FEF773
:10219000BDFD4FF480511948FEF7B8FD01201849E4
:1021A00008600020144908601648844217D16FF077
:1021B00001001449096808611248FFF757FE1248E8
:1021C00080881149C8800020888001F0A9FB4FF465
:1021D00080510E48FEF792FD08B901F0ABFE10BD2C
:1021E000C0000020000000200800002004000020A3
:1021F000100000200C00002018000020000C0140FE
:102200001400002008010020DC010020000801402B
:1022100070477047704700002DE9F84F044620686A
:1022200005682068C668206847694FF00009CA46FB
:1022300005F00F09B9F1000F0AD105F0200038B1FF
:1022400006F0200020B1204600F08DFEBDE8F88F9A
:10225000B9F1000F7BD007F0010018B906F49070B7
:10226000002874D005F0010030B106F4807018B178
:10227000606C40F00100606405F0040030B107F0CC
:10228000010018B1606C40F00200606405F00200CB
:1022900030B107F0010018B1606C40F004006064D8
:1022A00005F0080048B106F0200010B907F0010061
:1022B00018B1606C40F008006064606C002845D084
:1022C00005F0200028B106F0200010B1204600F0F3
:1022D0004AFE20684069C0F3801A606C00F0080074
:1022E00010B9BAF1000F2CD0204600F0E3FD2068B1
:1022F000406900F0400000B300BF00BF2168143106
:1023000051E8001F21F040002168143141E800022B
:10231000002AF3D100BFE06B50B17748E16B48630E
:10232000E06BFEF7B3F988B1E06B416B88470DE0D5
:102330002046FFF76FFF09E009E02046FFF76AFF3C
:1023400004E02046FFF766FF002060647EE7206B14
:10235000012877D105F01000002873D006F0100096
:102360000028FAD000BF002000902068006800908C
:1023700020684068009000BF00BF2068406900F0FE
:10238000400000285FD0E06B006840681FFA80F8CA
:10239000B8F1000F55D0A08D404552DDA4F82E8035
:1023A000E06B8069202843D000BF00BF21680C315A
:1023B00051E8001F21F4807021680C3141E80002CF
:1023C000002AF3D100BF00BF00BF2168143151E8DB
:1023D000001F21F001002168143141E80002002AA9
:1023E000F3D100BF00BF00BF2168143151E8001FC6
:1023F00021F040002168143141E80002002AF3D1A5
:1024000000BF202084F842000020206300BF00BFEE
:1024100021680C3151E8001F21F0100021680C31B7
:1024200041E80002002AF3D100BFE06BFEF702F999
:1024300002206063A08DE28D801A81B22046FFF7F2
:10244000E8FE03E742E0A08DE18D401A1FFA80F814
:10245000E08DD0B3B8F1000F37D000BF00BF2168C6
:102460000C3151E8001F21F4907021680C3141E8D3
:102470000002002AF3D100BF00BF00BF2168143161
:1024800051E8001F21F001002168143141E80002E9
:10249000002AF3D100BF202084F8420000202063EE
:1024A00000BF00BF21680C3151E8001F21F010006F
:1024B00021680C3141E80002002AF3D100BF02205C
:1024C000606341462046FFF7A4FEBFE605F08000AA
:1024D00030B106F0800018B1204600F061FEB5E68C
:1024E00005F0400030B106F0400018B1204600F081
:1024F00017FDABE600BFA9E6EB2D000810B50446BA
:102500000CB9012010BDA06900B100E000BF94F833
:10251000410028B9002084F84000204600F02AF845
:10252000242084F841002068C06820F4005021680D
:10253000C860204600F096FD2068006920F49040B5
:10254000216808612068406920F02A0021684861FC
:102550002068C06840F400502168C86000206064B2
:10256000202084F8410084F842000020606300BF0E
:10257000C8E7000010B586B0044600200290039022
:10258000049005902A49206888424FD100BF29480D
:10259000806940F48040274988610846806900F4DA
:1025A0008040019000BF00BF00BF0846806940F036
:1025B000040088610846806900F00400019000BFB3
:1025C00000BF48150290022003900320059002A945
:1025D0001948FEF703FA4FF4806002900020039040
:1025E000049002A91448FEF7F9F914481449086048
:1025F000102048600021124881608021C1600021C4
:10260000016141618161C161FEF766F908B1FDF7C1
:10261000C2FF00BF0A48A063446200BF0022114607
:102620002520FEF709FC2520FEF7F6FB06B010BDBD
:102630000038014000100240000801404400024000
:102640009801002070B504460D46164694F84200E5
:1026500020280BD105B10EB9012070BD00202063E8
:1026600032462946204600F07BFDF6E70220F4E7DB
:1026700010B5044603492068884201D101F09CF955
:1026800010BD0000003801402DE9F84F04460E4609
:10269000174699464FF0000A94F84100202850D17F
:1026A00006B117B90120BDE8F88F00206064212031
:1026B00084F84100FEF73AFB8246A784E784A068CD
:1026C000B0F5805F04D1206910B90025B04602E062
:1026D00035464FF000081EE0534600228021204678
:1026E000CDF8009000F08CFD20B1202084F841004E
:1026F0000320D8E745B9B8F80000C0F30800216806
:10270000486008F1020803E02878216848606D1CE1
:10271000E08C401EE084E08C0028DDD1534600228E
:1027200040212046CDF8009000F06AFD20B1202025
:1027300084F841000320B6E7202084F841000020FF
:10274000B1E70220AFE70000F7B50446154694F85C
:102750004100202836D1019800B10DB90120FEBDFD
:1027600001982062A584E58400206064212084F81B
:1027700041001548A16B88621448A16BC8621448D7
:10278000A16B08630020A16B486301AE23681A1D8A
:1027900031682B46A06BFEF7D3F86FF0400021683C
:1027A000086000BF00BF2168143151E8001F41F0EC
:1027B00080002168143141E80002002AF3D100BFF3
:1027C0000020CCE70220CAE74F2E0008A72E000801
:1027D000FF2D00087047704700BFFEE708B500BF37
:1027E0000A48406940F001000849486108464069CC
:1027F00000F00100009000BF00BF002211460E2033
:10280000FEF71AFB0E20FEF707FB08BD0010024082
:1028100000B585B00020019002900390049000BFA5
:102820003248806940F0200030498861084680695C
:1028300000F02000009000BF00BF00BF0846806984
:1028400040F0040088610846806900F004000090B0
:1028500000BF00BF00BF0846806940F008008861E3
:102860000846806900F00800009000BF00BF002209
:1028700042F202011E48FEF753FA012211031C48DE
:10288000FEF74EFA0122D1021A48FEF749FA01205A
:10289000019000200290039001A91548FEF79EF8D0
:1028A00043F20200019001200290002003900220D8
:1028B000049001A90E48FEF791F84FF400600190D2
:1028C00001200290002003900220049001A90948F1
:1028D000FEF784F84FF4805001900020029003909E
:1028E00001A90448FEF77AF805B000BD00100240C7
:1028F000000C01400008014010B50E480E49086068
:102900004FF48270486000210B488160C160016112
:1029100001214161890481613021C161002101628D
:10292000416281620A21C162FEF72EFE08B1FDF705
:1029300032FE10BD003001406800002000B587B0B5
:102940000020039004900590069001900290154895
:10295000154908604720486000211348816040F213
:10296000E731C1600021016141618161FFF7D0F968
:1029700008B1FDF710FE4FF48050039003A90A48F8
:10298000FFF793FA08B1FDF706FE002001900290D0
:1029900001A90548FFF77AF908B1FDF7FCFD07B07A
:1029A00000BD0000002C0140C000002000B587B031
:1029B0000020039004900590069001900290144826
:1029C000144908604720486000211248816040F2A5
:1029D000E731C160002101618161FFF799F908B118
:1029E000FDF7D9FD4FF48050039003A90948FFF784
:1029F0005CFA08B1FDF7CFFD00200190029001A91B
:102A00000448FFF743F908B1FDF7C5FD07B000BD65
:102A1000000400400801002010B50B480B49086075
:102A20004FF4FA204860002108488160C1600161CC
:102A30000C21416100218161C161FFF75FFD08B197
:102A4000FDF7A9FD10BD0000003801405001002035
:102A500000BFFEE730B502464FF6FF7012B10446E4
:102A6000A14200D130BD11E012F8014B60400023BB
:102A70000AE000F0010424B140104AF20104604071
:102A800000E040105C1CE3B2082BF2DB0C00A1F16B
:102A90000105A9B2E8D100BFE4E700BFFEE7704737
:102AA00008B508490968C9084FF47A72B1FBF2F118
:102AB0004143009100BF00BF00994A1E00920029C7
:102AC000F9D108BD3C000020F8B504460E46154675
:102AD0006068B0F5827F0DD1A068B0F5004F03D0DB
:102AE000A068B0F5806F05D12068006820F0400034
:102AF000216808606068B0F5827F11D1A068B0F5E8
:102B0000806F0DD13346002201212046009500F050
:102B100039F898B1606D40F0200060650320F8BD81
:102B20003346002280212046009500F02BF828B182
:102B3000606D40F0200060650320F0E70020EEE7C4
:102B4000F8B504460E4615463346012202212046BA
:102B5000009500F017F828B1606D40F02000606526
:102B60000320F8BD3346002280212046009500F066
:102B700009F828B1606D40F0200060650320F0E79F
:102B80000020EEE72DE9F84F04460D4690461E461C
:102B9000DDF82890FEF7CAF8A0EB0900371AFEF717
:102BA000C5F882462C480068C0F3CB3078430090CB
:102BB00045E0701C002842D0FEF7B8F8A0EB0A00F0
:102BC000B84200D2A7BB2068406820F0E00021682E
:102BD00048606068B0F5827F0DD1A068B0F5004F05
:102BE00003D0A068B0F5806F05D12068006820F0A0
:102BF000400021680860A06AB0F5005F0DD100BFF9
:102C00002068006820F4005021680860206800688F
:102C100040F400502168086000BF012084F8510092
:102C200000BF002084F8500000BF0320BDE8F88FEB
:102C3000FFE7009800B900270098401E0090206828
:102C400080682840A84201D1012000E000204045D2
:102C5000AFD10020EAE700003C000020704710B52B
:102C6000FEF76AF810BD00B58FB0282105A8FDF762
:102C7000F2FA14216846FDF7EEFA012005900004EF
:102C80000690002007900120099002200C90C103BB
:102C90000D914FF4E0110E9105A8FEF743FA08B12B
:102CA000FDF779FC0F200090022001900020029097
:102CB0004FF4806003900020049002216846FEF7E4
:102CC0000DF908B1FDF767FC0FB000BD70470000BB
:102CD00010B50248FFF770F910BD0000C0000020D9
:102CE00010B50248FFF768F910BD00000801002088
:102CF00010B502681C4B984208D0B0F1804F05D047
:102D00001A4B984202D01A4B984203D122F070021B
:102D10004B681A43144B984208D0B0F1804F05D04D
:102D2000124B984202D0124B984203D122F44072C7
:102D3000CB681A4322F080034C6943EA0402026024
:102D40008B68C3620B688362074B984201D10B69A1
:102D5000036301234361036903F001031BB10369AA
:102D600023F00103036110BD002C0140000400406A
:102D70000008004030B50C46816821F47F4142EAEA
:102D8000032525432943816030BD0A46816821F02F
:102D9000700142F0070319438160704730B50B465C
:102DA0001446026A056A25F001050562816921F071
:102DB000F00141EA041122F00A021A438161026221
:102DC00030BD30B50B461446026A056A25F0100581
:102DD0000562816921F4704141EA043122F0A002C8
:102DE00042EA03128161026230BD70B505466C6A29
:102DF0000020E085E0842046FFF70CFA70BD70B536
:102E000006460025746A20684069C0F3C01594F82E
:102E10004100212805D125B10020E084204600F0A2
:102E20008FF820684069C0F3801594F8420022288A
:102E300005D125B10020E085204600F03BF8606C0C
:102E400040F0100060642046FFF7E4F970BD70B5F3
:102E500005466C6A2868006800F02000F8B9002078
:102E6000E08400BF00BF2168143151E8001F21F049
:102E700080002168143141E80002002AF3D100BF2C
:102E800000BF00BF21680C3151E8001F41F0400035
:102E900021680C3141E80002002AF3D102E020460B
:102EA000FFF798FC70BD70B50446656A2846FFF7C9
:102EB00092FC70BD00BF00BF02680C3252E8002FC8
:102EC00022F4907102680C3242E80013002BF3D117
:102ED00000BF00BF00BF0268143252E8002F22F08A
:102EE00001010268143242E80013002BF3D100BF45
:102EF000016B01290ED100BF00BF02680C3252E8FD
:102F0000002F22F0100102680C3242E80013002B5F
:102F1000F3D100BF202180F84210002101637047E7
:102F200010B504462068C06820F040002168C860E1
:102F3000202084F841002046FFF74CFC002010BD03
:102F400000BF00BF02680C3252E8002F22F0C0011F
:102F500002680C3242E80013002BF3D100BF20219D
:102F600080F841107047F8B5044694F842002228D2
:102F700075D1A068B0F5805F0CD1206950B90025EB
:102F8000A66A20684068C0F308003080A06A801CF0
:102F9000A06215E0A56A0026A068B0F5805F03D0A6
:102FA000A06828B9206918B920684068287004E032
:102FB0002068406800F07F002870A06A401CA06272
:102FC000E08D401E80B2E085002846D12068C068B0
:102FD00020F020002168C8602068C06820F480705C
:102FE0002168C8602068406920F0010021684861BC
:102FF000202084F8420000206063206B012826D145
:103000000020206300BF00BF21680C3151E8001F81
:1030100021F0100021680C3141E80002002AF3D1B0
:1030200000BF2068006800F0100010280AD100BF1F
:1030300000200090206800680090206840680090A0
:1030400000BF00BFA18D2046FFF7E3F802E0204655
:10305000FFF70EFB0020F8BD01E00020FBE7022097
:10306000F9E7000070B504462168096921F4405170
:10307000E2681143226811612269A1681143626903
:1030800041EA02052168C96841F20C629143294373
:103090002268D1602168496921F44071A269114315
:1030A000226851612D4A2168914202D1FDF7F2FF59
:1030B00001E0FDF7DFFF00EBC00101EB00116268EA
:1030C0009200B1FBF2F100EBC00202EB0012636868
:1030D0009B00B2FBF3F26423B2FBF3F202EBC203F8
:1030E00003EB0212A1EB8201322202EB01116422F6
:1030F000B1FBF2F101F0F00100EBC00202EB0012B3
:1031000063689B00B2FBF3F26423B2FBF3F201EBC2
:10311000021200EBC00101EB001163689B00B1FBE0
:10312000F3F100EBC00303EB00136668B600B3FBDA
:10313000F6F36426B3FBF6F303EBC30606EB0313C7
:10314000A1EB8301322303EB01116423B1FBF3F103
:1031500001F00F0111442268916070BD00380140F8
:1031600010B5034699629A85DA85002058642220BA
:1031700083F84200186928B11868C06840F480706C
:103180001C68E0601868406940F001001C686061DC
:103190001868C06840F020001C68E060002010BD86
:1031A000014691F84100212828D18868B0F5805F58
:1031B0000BD1086948B90A6A1088C0F308000B6887
:1031C0005860086A801C086205E00B6A581C086297
:1031D00018780B685860C88C401E80B2C88458B9F3
:1031E0000868C06820F080000B68D8600868C06874
:1031F00040F040000B68D860002070470220FCE7D8
:103200002DE9F84304460D4617469846089E31E0DE
:10321000701C70B3FDF78AFDA0EB0800B04200D827
:1032200016B90320BDE8F8832068C06800F00400E8
:10323000F8B1802D1ED0402D1CD020680068C0F34E
:10324000C000B0B100BF002000902068006800906E
:1032500020684068009000BF00BF2046FFF72AFEAC
:103260000820606400BF002084F8400000BF0120F7
:10327000D8E7FFE7206800682840A84201D1012074
:1032800000E00020B842C3D00020CBE710B50248D0
:10329000FEF7C2FF10BD00005001002000BFFEE796
:1032A0000246024B23F8121070470000C6020020AD
:1032B00070B50A46B2F57F4F19D1A0F11001CC17B5
:1032C00001EB5474E410174D2C5D0B46DD1703EB36
:1032D0005575ED10A3EBC5060125B5402C43E5B2AD
:1032E000CC1701EB5474E4100E4E355518E0BAB902
:1032F000A0F11001CC1701EB5474E410094D2C5DC2
:103300000B46DD1703EB5575ED10A3EBC506012544
:10331000B540AC43CD1701EB5575ED10014E74551A
:1033200070BD0000F001002002480068C0F30220D8
:10333000704700000CED00E010B5002804DB0A0720
:10334000130E054A135406E00A07140E034A00F050
:103350000F031B1FD45410BD00E400E018ED00E083
:1033600000BF70472DE9F041F648006808283ED2BA
:10337000DFE800F0043E79B3F1EFEEED0120FCF759
:10338000F5FF06460022F04B01F074F8044601F008
:103390002DF8EC49096801EB8101EC4A02EB81014F
:1033A000EB4A126821F8120000200EE0E549096896
:1033B00001EB8101E54A02EB810131F81010E54A89
:1033C00012681144E34A1160401C0A28EEDBE14810
:1033D00000680A2190FBF1F0DF49DA4A126821F80F
:1033E00012000020DB4908600120D6490860A5E1F1
:1033F0000220FCF7BBFF06460022D34B01F03AF84F
:10340000044600F0F3FFCF49096801EB8101CF4A80
:1034100002EB8101CE4A126821F8120000200EE072
:10342000C849096801EB8101C84A02EB810131F802
:103430001010C84A12681144C64A1160401C0A287C
:10344000EEDBC44800680A2190FBF1F081B2C2486B
:10345000BC4A126820F812100020BE490860022001
:10346000B84908606AE10320FCF780FF06460022A5
:10347000B54B00F0FFFF044600F0B8FFB149096802
:1034800001EB8101B14A02EB8101B14A126821F8D6
:10349000120000200EE0AB49096801EB8101AB4A44
:1034A00002EB810131F81010AA4A12681144A94AAE
:1034B0001160401C0A28EEDBA64800680A2190FB38
:1034C000F1F0A5499F4A126821F812000020A14995
:1034D000086003209B49086030E10420FCF746FFA8
:1034E00006460022984B00F0C5FF044600F07EFF20
:1034F0009449096801EB8101944A02EB8101944AE5
:10350000126821F8120000200EE08E49096801EBD4
:1035100081018E4A02EB810131F810108D4A126848
:1035200011448C4A1160401C0A28EEDB894800686F
:103530000A2190FBF1F08849824A126821F81200B2
:1035400000208449086004207E490860F6E0B1E06C
:1035500075E03AE0FFE70520FCF708FF0646002289
:10356000794B00F087FF044600F040FF7549096879
:1035700001EB8101754A02EB8101754A126821F85D
:10358000120000200EE06F49096801EB81016F4ACB
:1035900002EB810131F810106E4A126811446D4A35
:1035A0001160401C0A28EEDB6A4800680A2190FB83
:1035B000F1F06949634A126821F812000020654958
:1035C000086005205F490860B8E00620FCF7CEFEE1
:1035D000064600225C4B00F04DFF044600F006FF5B
:1035E0005849096801EB8101584A02EB8101584AA8
:1035F000126821F8120000200EE05249096801EB20
:103600008101524A02EB810131F81010514A1268CF
:103610001144504A1160401C0A28EEDB4D480068F6
:103620000A2190FBF1F04C49464A126821F8120039
:103630000020484908600620424908607EE00720D3
:10364000FCF794FE064600223F4B00F013FF0446B1
:1036500000F0CCFE3B49096801EB81013B4A02EBDB
:1036600081013B4A126821F8120000200EE0354922
:10367000096801EB8101354A02EB810131F8101034
:10368000344A12681144334A1160401C0A28EEDBA8
:10369000304800680A2190FBF1F081B22E48294A97
:1036A000126820F8121000202A49086007202549D6
:1036B000086043E00020FCF759FE06460022224B3A
:1036C00000F0D8FE044600F091FE1E49096801EBA7
:1036D00081011E4A02EB81011D4A126821F8120085
:1036E00000200EE01749096801EB8101174A02EB3F
:1036F000810131F81010174A12681144154A1160FF
:10370000401C0A28EEDB134800680A2190FBF1F008
:1037100011490C4A126821F8120000200D49086076
:10372000084908600A480068401C094908600846C2
:103730000068092801DD0020086000BF00BFBDE867
:10374000F08100006000002000002440460C0020B2
:103750005C000020580000200602002010B5012265
:1037600002210C48FDF7DCFA06210020FCF7B8FE28
:1037700008210120FCF7B4FE00210220FCF7B0FE76
:10378000D0210320FCF7ACFE00210420FCF7A8FEAA
:1037900010BD0000000C0140FDF7DAFAFFF763FAF4
:1037A000FFF736F8FFF71AF8FFF7A6F8FFF734F936
:1037B000FFF7C4F8FFF7FAF80848FEF71BFB00F024
:1037C000D1F8FFF7CBFF07E00548006820B1FFF70D
:1037D000C9FD002002490860F6E70000C000002093
:1037E000000000202DE9F04104460D460CB1022DE9
:1037F00001DABDE8F08126786778284800688642BB
:1038000001D0002E48D1052F3AD008DC012F0DD071
:10381000022F11D0032F15D0042F37D118E0062F17
:103820001CD00F2F20D0102F30D123E0A81E81B242
:10383000A01C00F009F92EE0A81E81B2A01C00F027
:10384000B9F928E0A81E81B2A01C00F065FA22E0B8
:10385000A81E81B2A01C00F0E7FA1CE0A81E81B2ED
:10386000A01C00F061FD16E0A81E81B2A01C00F0B3
:10387000B1FB10E0A81E81B2A01C00F063FC0AE0BE
:10388000A81E81B2A01C00F0E7FC04E060780121D2
:1038900000F006F800BF00BF00BFAAE7400000200C
:1038A000F0B5ADF2044D05460E4600240027194838
:1038B00002782146641C01A8425445F0800221464A
:1038C000641C42542146641C46542146FFF7C2F84A
:1038D00007462146641C01A847543A122146641C3D
:1038E00042540D48008AA04201DB204601E00A480C
:1038F000008A094948824A8AC86801A9FCF766FC1F
:103900000548428AC168054800F05AFB0DF2044D93
:10391000F0BD000040000020DC010020500100202C
:103920002DE9F04100240E480568C488022C01DA14
:10393000BDE8F081A01E295C601E285C41EA0027DA
:10394000A01E81B22846FFF785F80646B74200D090
:10395000EEE7034AD1881068FFF744FF00BFE7E7AE
:10396000DC01002010B50E480E4908600020888058
:10397000C88008720C48C8604FF48060088200203C
:103980004882012209490A48FEF75CFE6FF00100F7
:103990000849096808610748FEF72CFA10BD0000C5
:1039A00046040020DC010020460800201C00002006
:1039B000500100200801002010B51B48808840F20B
:1039C000FF3188420EDB00201749888008460068D6
:1039D000002101604FF6FF730A2214A11648FEF77A
:1039E00053FE1AE0154800780F498988144A50544C
:1039F000124801780C4882888088401C0A4B9880C5
:103A00001846006881540F48FEF730FA00200D492F
:103A1000096848620B48FEF7EDF90122074906489C
:103A2000FEF710FE10BD0000DC010020CAFDBEDD67
:103A3000D2E7B3F600000000500100201C00002077
:103A400046040020080100202DE9F04FADF2144D8E
:103A5000054600240020CDF804044FF4806101A83D
:103A6000FCF7F9FB6878297840EA0129E878A97819
:103A700040EA0126012E01DA502E72DCB9F15F0F07
:103A800070DC06EB09006028FADCF01DC11700EBC2
:103A90005171C1F3C701CDF8101443480278204694
:103AA000611CCCB201A90A5401222046611CCCB28F
:103AB00001A90A542146621CD4B201AADDF81004FF
:103AC00050540027BB462FE0002001A9085582462C
:103AD0001BE009EB070188B20DF20C41FCF772FD07
:103AE00001A8005D9DF80C1401FA0AF1084301A930
:103AF0000855781C87B2B74203DB0120CDF80404D7
:103B000006E00AF1010000F0FF0ABAF1080FE0DB5D
:103B100000BF601CC4B2DDF80404012800D107E036
:103B20000BF1010000F0FF0BDDF810048345CBDB47
:103B300000BF214601A8FEF78DFF80462046611C8C
:103B4000CCB201A901F800804FEA28222046611C6E
:103B5000CCB201A90A541548008AA04203DB2046D2
:103B600003E017E012E01148008A104948824A8AAF
:103B7000C86801A9FCF72AFB0C48428AC1680C48B6
:103B800000F01EFA0DF2144DBDE8F08F0220CDF8C2
:103B9000080402E00320CDF808040120DDF8081431
:103BA000FFF77EFE00BFEDE740000020DC010020B3
:103BB000500100202DE9F04FADF2144D05460024D0
:103BC0000020CDF804046878297840EA0129E878D3
:103BD000A97840EA0126012E01DA602E72DCB9F1E3
:103BE0005F0F70DC06EB09006028FADCF01DC117DE
:103BF00000EB5171C1F3C701CDF8101443480278AE
:103C00002046611CCCB201A90A5402222046611C44
:103C1000CCB201A90A542146621CD4B201AADDF833
:103C2000100450540027BB462FE0002001A908557E
:103C300082461BE009EB070188B20DF20C41FCF74C
:103C4000DDFC01A8005D9DF80C1401FA0AF108439F
:103C500001A90855781C87B2B74203DB0120CDF8D3
:103C6000040406E00AF1010000F0FF0ABAF1080FAF
:103C7000E0DB00BF601CC4B2DDF80404012800D101
:103C800007E00BF1010000F0FF0BDDF810048345A5
:103C9000CBDB00BF214601A8FEF7DCFE80462046B4
:103CA000611CCCB201A901F800804FEA282220460D
:103CB000611CCCB201A90A541548008AA04203DB5A
:103CC000204603E017E012E01148008A10494882BC
:103CD0004A8AC86801A9FCF779FA0D48428AC16886
:103CE0000C4800F06DF90DF2144DBDE8F08F022084
:103CF000CDF8080402E00320CDF808040220DDF826
:103D00000814FFF7CDFD00BFEDE7000040000020E4
:103D1000DC010020500100202DE9F04FADF2044DF0
:103D2000064600241EB90DF2044DBDE8F08F7078F0
:103D3000317840EA0127F078B17840EA0125012D79
:103D400064DB602D62DC5F2F5DDC781900285ADBB4
:103D50007819602857DC314802782046611CCCB2C3
:103D600001A90A5403222046611CCCB201A90A54BD
:103D70006806020E2046611CCCB201A90A544FF01D
:103D8000000816E007EB080188B2FCF707FC814643
:103D90004FEA29222046611CCCB201A90A542046D0
:103DA000611CCCB201A901F8009008F101001FFAD2
:103DB00080F8A845E6DB214601A8FEF74BFE8246C7
:103DC0002046611CCCB201A901F800A04FEA2A22CA
:103DD0002046611CCCB201A90A541148008AA042B5
:103DE00001DB204601E00E48008A0D4948824A8ADC
:103DF000C86801A9FCF7EAF90948428AC16809487C
:103E000000F0DEF88FE74FF0020B01E04FF0030BFC
:103E100059460320FFF744FD00BF84E7400000201F
:103E2000DC010020500100202DE9F04FADF2044DDF
:103E3000054600241DB90DF2044DBDE8F08F6878E9
:103E4000297840EA0127E878A97840EA0126012E7E
:103E500061DB602E5FDC5F2F5ADCB819602857DC0D
:103E6000314802782046611CCCB201A90A540422D0
:103E70002046611CCCB201A90A547006020E2046ED
:103E8000611CCCB201A90A544FF0000816E007EB00
:103E9000080188B2FCF78CFB81464FEA29222046B4
:103EA000611CCCB201A90A542046611CCCB201A904
:103EB00001F8009008F101001FFA80F8B045E6DB38
:103EC000214601A8FEF7C6FD82462046611CCCB201
:103ED00001A901F800A04FEA2A222046611CCCB2B9
:103EE00001A90A541148008AA04201DB204601E0E2
:103EF0000E48008A0D4948824A8AC86801A9FCF721
:103F000065F90A48428AC168094800F059F892E701
:103F10004FF0020B01E04FF0030B59460420FFF76E
:103F2000BFFC00BF87E7000040000020DC0100204C
:103F30005001002010B51C48006830B100224FF439
:103F400000611A48FCF7ECFE2DE019480068007883
:103F5000EE2828D116480068407820BB012012497D
:103F6000086013480068807900EB8000401D11490B
:103F700008600F4800688079401C0F4988710C4820
:103F80000068807888700A480068C078C87008485F
:103F90000068007908710648006840794871072276
:103FA000064800F00DF810BD200000200008014078
:103FB000DC010020400000202400002050010020EF
:103FC00070B504460D461646324629462046FEF791
:103FD000BBFB70BD2DE9F04FADF2144D044600253A
:103FE0000020CDF804046078217840EA012AE078C6
:103FF000A17840EA01262079CDF80C04012E78DB67
:10400000502E76DCDDF80C04C000B042F7DBBAF1CC
:104010005F0F6FDC0AEB060060287FDC0027A946F3
:1040200036E009F10500205CCDF808044FF0000BE4
:1040300021E0012000FA0BF0DDF80814084020B15F
:104040004FF47F40CDF8100402E00020CDF81004BA
:104050000AEB070188B2DDF81014FFF729F9781C84
:1040600087B2B74203DB0120CDF8040406E00BF170
:10407000010000F0FF0BBBF1080FDADB00BFDDF839
:104080000404012800D107E009F1010000F0FF0954
:10409000DDF80C048145C4DB00BF274802782846C0
:1040A000691CCDB20DF800200F222846691CCDB244
:1040B0000DF800200DEB050021680160281DC5B238
:1040C00029466846FEF7C6FC804608F0FF022846EF
:1040D000691CCDB20DF800204FEA28222846691C41
:1040E000CDB20DF800201548008AA84203DB28460F
:1040F00003E017E012E01148008A104948824A8A1A
:10410000C8686946FCF762F80C48428AC1680C48E6
:10411000FFF756FF0DF2144DBDE8F08F0220CDF8E9
:10412000000402E00320CDF800040F20DDF80014A5
:10413000FFF7B6FB00BFEDE740000020DC010020E8
:10414000500100202DE9F04FADF2044D0446002649
:104150001CB90DF2044DBDE8F08F6078217840EA7B
:104160000128E078A17840EA012794F804B0012FF3
:1041700063DB602F61DCBBEB470F5ED1B8F15F0FF3
:1041800058DC08EB0700602854DC002514E006200A
:1041900000EB4500205C052101EB4501615C40EA34
:1041A0000120CDF8000408EB050188B2DDF8001409
:1041B000FFF776F8681C85B2BD42E8DB2348027839
:1041C0003046711CCEB20DF8002010223046711C12
:1041D000CEB20DF800200DEB060021680160301D05
:1041E000C6B231466846FEF735FC814609F0FF024B
:1041F0003046711CCEB20DF800204FEA292230461D
:10420000711CCEB20DF800201148008AB04201DBCB
:10421000304601E00E48008A0D4948824A8AC86843
:104220006946FBF7D3FF0A48428AC1680948FFF78D
:10423000C7FE8EE74FF0020A01E04FF0030A0AF0D2
:10424000FF011020FFF72CFB00BF82E74000002099
:10425000DC010020500100202DE9F047ADF5806D14
:1042600005468A4600246878297840EA0129E878DA
:10427000A97840EA012717B1B7F57F4F46D1B9F1C8
:104280005F0F40DC39464846FFF712F823480278B2
:104290002046611CCCB20DF8002005222046611C8E
:1042A000CCB20DF800200DEB040029680160201D40
:1042B000C4B221466846FEF7CDFB0646F2B2204660
:1042C000611CCCB20DF8002032122046611CCCB229
:1042D0000DF800201248008AA04201DB204601E0D0
:1042E0000F48008A0E4948824A8AC8686946FBF727
:1042F0006DFF0B48428AC1680A48FFF761FE0DF561
:10430000806DBDE8F0874FF0020801E04FF0030830
:1043100041460520FFF7C4FA00BFF0E74000002047
:10432000DC010020500100202DE9F047ADF5806D43
:1043300005468A4600241DB90DF5806DBDE8F0875D
:104340006878297840EA0127E878A97840EA0128C6
:104350005F2F3DDC41463846FEF7A2FF2048027839
:104360002046611CCCB20DF8002006222046611CBC
:10437000CCB20DF800200DEB040029680160201D6F
:10438000C4B221466846FEF765FB0646F2B22046F7
:10439000611CCCB20DF8002032122046611CCCB258
:1043A0000DF800200F48008AA04201DB204601E002
:1043B0000C48008A0B4948824A8AC8686946FBF75C
:1043C00005FF0848428AC1680748FFF7F9FDB3E7CF
:1043D0004FF0020949460620FFF762FA00BFABE73B
:1043E00040000020DC010020500100204FEA115362
:1043F000A3F58063D3F11E03A8BFD3F1200C08DB23
:104400004FF0004242EAC12252EA505232FA03F01F
:10441000704709420BD4102BC4BF0020704703F52E
:10442000787CBCF1FF3F05D04FF0FF3070474FF074
:104430000000704770B500F0C7F800BF49922480B3
:1044400000207047F0E710F0004248BF4042B0FA49
:1044500080F310FA03F10AD0C3F11D0303F5806362
:104460004FEA415002EB035202EBD12170474FF06B
:1044700000007047DFF848C170B51CEA111E1EBF6E
:104480001CEA13159EEA0C0F95EA0C0F00F06F80E2
:1044900081EA030423EA4C134EEAD47E21EA4C114C
:1044A00041F4801143F48013AE44A1FB024CA0FB05
:1044B0000365AEF17F7E361955EB0C05A1FB034C6D
:1044C0004CF10003A0FB021C16EB0C06654153F1F6
:1044D0000003094218BF46F0010613F4007F0BD118
:1044E0004FEA03314FEA0530340341EA155140EAFF
:1044F00016506FF003020AE04FEAC3214FEAC520CD
:10450000F40241EA555140EA56506FF0020202EBC4
:104510002E4201EB025585EACE710AD05FEA440CC7
:1045200018BF24F0004450F1000041F1000120EADE
:10453000D47040F2FE7C624500D270BDA84214BF28
:104540004FF080444FF04044002E08BF0024BEF1DD
:10455000806FA8BFA1F1C041BDE8704080F28280A9
:104560004FF0000001F1C04101F0004170479EEAA8
:104570000C0F0CEA131518BF95EA0C0F06D04FF07C
:10458000000081EA030E0EF0004170BD00F01CF83F
:104590008900013E00F007B800F009B84FEA430C6B
:1045A0005FEA5C5C08D081EA030100F05BB84FEA87
:1045B000410C5FEA5C5CF6D14FF0000001497047A6
:1045C0000000FF070000F87F0EF1020E2EF0030E30
:1045D0005EF8046B364205D4012A43EB030515F55A
:1045E000001F12D8012841EB010C1CF5001F0CD84C
:1045F0000ED14FEAD17C15F5001F0CEB4C0C0CF1E1
:10460000020C08BF4CEBD37C04E04FF0080C01E037
:104610004FEAD37C0CEB4C0526FA05F606F00706AC
:10462000B6F1040C06D20EEB860CBDE870404CF0DF
:10463000010C6047DFE80CF0090B02024FF000416B
:104640004FF00000A1F5002170BD19461046012869
:1046500051EB010418BFD4F5001484BF002001F011
:10466000004170BD0808A0F500114FEA3101704704
:1046700002030405060708090A0B0C0D0E0F1010A3
:104680000102000000000000000001020304060710
:10469000080900000000010203040000BC460008F5
:1046A00000000020680000002801000824470008DE
:1046B00068000020E0120000440100080000000033
:1046C00000000000000000000000000000000000EA
:1046D00000000000000000000000000000000000DA
:1046E000EE010000000000000000000000000000DB
:1046F000100000000100000000127A000500000018
:1047000000000000000000000000000000000000A9
:104710000000000000000000000000000000000099
:044720000000000095
:04000005080000ED02
:00000001FF
